:020000040800F2
:1000000000040020E1010008590E00085D0E000800
:10001000B10E00085D0E0008850E0008E30100081F
:10002000E3010008E3010008E3010008692F00086C
:10003000E3010008E3010008E3010008E301000810
:10004000E3010008E3010008E3010008E301000800
:10005000E3010008E3010008CD310008F931000890
:1000600025320008513200087D320008E301000803
:10007000E3010008E3010008E3010008E3010008D0
:10008000E3010008E3010008E3010008E3010008C0
:10009000E3010008E3010008E3010008A9320008B9
:1000A000E3010008E3010008E3010008E3010008A0
:1000B000E3010008E3010008E3010008E301000890
:1000C000E3010008E3010008E3010008E301000880
:1000D000E3010008E3010008E3010008E301000870
:1000E00011330008E3010008E3010008E301000800
:1000F000E3010008E3010008E3010008E301000850
:10010000E3010008E3010008E52F0008E30100080F
:10011000E3010008E3010008E3010008E30100082F
:10012000E3010008E3010008E3010008E30100081F
:10013000E3010008E3010008E3010008E30100080F
:10014000E3010008E3010008E3010008B12600080C
:10015000E3010008E3010008E3010008E3010008EF
:10016000E3010008E3010008E3010008E3010008DF
:10017000E3010008E3010008E3010008E3010008CF
:10018000E3010008E3010008E3010008E3010008BF
:10019000E3010008E3010008E3010008E3010008AF
:1001A000E3010008E3010008E3010008E30100089F
:1001B000E3010008E3010008E3010008E30100088F
:1001C000E3010008E3010008E3010008E30100087F
:1001D000E3010008E3010008E3010008E30100086F
:1001E00002E000F000F8FEE772B6394880F30888B4
:1001F000384880F3098838484EF60851CEF200019D
:10020000086040F20000CCF200004EF63471CEF2ED
:1002100000010860BFF34F8FBFF36F8F40F2000003
:10022000C0F2F0004EF68851CEF200010860BFF334
:100230004F8FBFF36F8F4FF00000E1EE100A4EF6C4
:100240003C71CEF200010860062080F31488BFF3F1
:100250006F8F01F0F5FE02F01DFE4FF055301F4983
:100260001B4A91423CBF41F8040BFAE71C49194A6A
:1002700091423CBF41F8040BFAE71A491A4A1B4B5A
:100280009A423EBF51F8040B42F8040BF8E70020F5
:100290001749184A91423CBF41F8040BFAE701F0B4
:1002A000D3FE02F053FE144C144DAC4203DA54F862
:1002B000041B8847F9E700F03FF8114C114DAC42A0
:1002C00003DA54F8041B8847F9E701F0BBBE0000CD
:1002D000000400200024002000000008000000208E
:1002E00000040020203700080024002028240020DB
:1002F0002824002018340020E0010008E001000854
:10030000E0010008E00100082DE9F04F2DED108A12
:10031000C1F80CD0C3689D46BDEC108ABDE8F08FD3
:10032000002383F311882846A047002001F00EFB2C
:1003300001F0BEFA00DFFEE71A4B0C2270B5002474
:100340001A700F225C709C70DC701C715C719C7167
:10035000DC711C725C729A72DC7201F043FE06461C
:1003600001F068FE054650B90F4B9E4217D001338D
:100370009E4241F2883412BF054600240125002028
:1003800001F03AFE0DB100F0B5F800F039FD00F0D3
:1003900003FC204600F00CF900F0ACF8F9E7044645
:1003A000EDE700BF28240020010007B008B500F0E9
:1003B00095FBA0F120035842584108BD07B5054BF5
:1003C00002211B88ADF8043001A800F0D5FB03B072
:1003D0005DF804FBF4330008064991F8243033B18A
:1003E00000230822086A81F8243000F0F7BB0120BE
:1003F000704700BF482400202DE9F84F234C94F8A3
:1004000024300546884617468BBB2E46DFF87C9085
:10041000002F38D094F824A0BAF1000F05D1202283
:10042000FF214846266200F0D9FCCAF10805BD420A
:1004300028BF3D465FFA85FBAD0041462A4604EBE6
:100440008A0000F0A1FC94F82430A7EB0B079B4432
:100450005FFA8BFBBBF1080F2E44A844FFB284F86F
:1004600024B0D5D1FFF7B8FF0028D1D108E0266A23
:1004700006EB8306B042C9D0FFF7AEFF0028C4D117
:100480000020BDE8F88F0120BDE8F88F4824002047
:1004900010B5202383F311881248C3680BB101F013
:1004A000DBFA0023104A0F484FF47A7101F098FAF2
:1004B000002383F311880D4C236813B12368013B9B
:1004C0002360636813B16368013B6360084B1B786A
:1004D00033B9636823B9022000F042FC3223636021
:1004E00010BD00BF342400209104000878290020AA
:1004F0007024002010B5254B254953F8042F0132F4
:1005000000D110BD8B42F8D1224C234B22689A4275
:100510003AD9224B9B6803F1006303F580339A427A
:1005200032D2002000F052FB1D4B0220187000F068
:1005300007FC1C4B1A6C00221A64196E1A66196E9D
:10054000596C5A64596E5A665A6E5A6942F0800262
:100550005A615A6922F080025A615A691A6942F056
:1005600000521A611A6922F000521A611B6972B6B0
:100570000D4A0E4B13601B682268202181F31188FD
:100580009D4683F30888104710BD00BFFCFF00089C
:100590001C00010804000108FFFF000828240020B7
:1005A000702400200038024008ED00E0000001083F
:1005B0002DE9F04FB04C97B020228146FF210EA8C4
:1005C000A66800F00BFCAD4A1378A346A3B9AC486B
:1005D0000121C3601170202383F31188C3680BB11C
:1005E00001F03AFA0023A74AA5484FF47A7101F0C6
:1005F000F7F9002383F31188B9F1000F02D0A24B61
:10060000C3F80090A14BA04A00241C7054602546FA
:1006100027469846012000F093FBB9F1000F00F047
:100620002282994B1B68002B40F01D8217B0BDE859
:10063000F08F0220FFF7BAFE002840F00E82944BA4
:100640001B88ADF82430022109A800F095FAE1E7F3
:100650004FF47A7000F042FA031E0193EFDB0220A0
:10066000FFF7A4FE82460028E9D0019B581E04280B
:1006700000F2F581DFE800F0030D1013160016A854
:10068000052340F8343D042100F076FA5446002753
:1006900052E004217848F7E704217E48F4E704217A
:1006A0007D48F1E71C24204600F092FA04340990BA
:1006B000042109A800F060FA2C2CF4D1E6E7002D03
:1006C000BDD0002CBBD00220FFF770FE05460028ED
:1006D00000F0C781012000F079FA022088F80000BC
:1006E00000F02EFB0024E3B21846019300F07EFADE
:1006F000824648B1019B184600F088FA0134002870
:10070000F1D12C46654B9BE70123022088F800308D
:1007100000F004FB5646DBF808309E4206D2304615
:1007200000F056FA0130ECD10436F4E7564B0026BF
:1007300088F800605E602C4600F058FB1DB1002C6C
:1007400018BF4FF00009FFF739FE63E7002D3FF4B3
:1007500076AF002C3FF473AF022088F8000000F061
:10076000EFFA322000F0BAF9B0F1000AC0F2798154
:100770001AF0030540F07581DBF8082006EB0A0348
:10078000934200F26E81BAF5807F00F26A81444B99
:10079000019355450DDA4FF47A7000F09FF90290FD
:1007A000029A002AC0F25D81019B029AEA54013547
:1007B000EEE7C820FFF7FAFD0546002800F051815A
:1007C0001F2E11D8C6F12004544528BF54460EAB45
:1007D00026F0030022463249184400F0D5FA22469A
:1007E000FF212F4800F0FAFA4FEAAA0A5FFA8AF2CC
:1007F0002B493046FFF700FE0446002881D006EB67
:100800008A06054698E70220FFF7D0FD00283FF44E
:1008100016AFFFF7E1FD00283FF411AF002292462A
:10082000DBF808309A4259D21F2A1ED80E9B01339A
:100830001BD022F0030316A90B4453F8203C099364
:100840001848436883B3174800210DF1240E11F8AE
:100850000E3083EA0A03DBB2013150F82330042959
:1008600083EA1A2AF3D10432DAE71046019200F043
:10087000AFF9019A0990E3E72824002074250020AD
:1008800034240020910400087829002070240020DE
:10089000F63300082C24002030240020F833000810
:1008A000742400207825002019464FF0080E11F01E
:1008B000010F4FEA51011FBF81F06D4181F43801F2
:1008C00081F4034181F02001BEF1010EEFD140F827
:1008D00023100133B3F5807FE6D1B4E716A80421D5
:1008E00040F84CAD00F048F926E716A8002340F880
:1008F000343D642100F01CF900287FF4A0AE0220F2
:10090000FFF754FD00283FF49AAE099800F090F9E3
:1009100016AB43F8480D04211846E3E716A8002358
:1009200040F8343D642100F003F900287FF487AEDD
:100930000220FFF73BFD00283FF481AE099800F04C
:1009400085F916AB43F8440DE5E70220FFF72EFDCD
:1009500000283FF474AE00F07FF916AB43F8400D69
:10096000D9E70220FFF722FD00283FF468AE09A96D
:10097000142000F077F9824616A8042140F83CAD17
:1009800000F0FAF8514609A8ACE7322000F0A6F8CA
:10099000B0F1000AFFF653AE1AF0030F7FF44FAE2A
:1009A000DBF808200AEB070393423FF648AE02202B
:1009B000FFF7FCFC00283FF442AE2AF0030ABA44D9
:1009C000BA453FF4B9AE384600F002F90421089068
:1009D00008A800F0D1F80437F2E74FF47A70FFF777
:1009E000E5FC00283FF42BAEFFF7F6FC00283FF4AF
:1009F00089AE0E9B01330CD008220EA90020FFF710
:100A0000FBFC00283FF47EAE2022FF210EA800F060
:100A1000E5F9FFF7D3FC304800F09EFF06E616A884
:100A2000002340F8343D642100F082F8824600281B
:100A30007FF405AE0220FFF7B9FC00283FF4FFADBC
:100A4000FFF7BCFC41F2883000F086FF099800F007
:100A500001FAD14600F0CAF9DCE505466CE600274C
:100A6000EDE52546EBE5002000F038F80290029B0A
:100A7000002BFFF6D2AD012000F050F9029B213B84
:100A8000122B3FF6C7AD01A252F823F0330600083F
:100A900051060008BF0600081506000815060008E4
:100AA000150600084D0700088B0900080708000814
:100AB000EB0800081D0900084B090008150600088E
:100AC0006309000815060008DB090008390700085B
:100AD000150600081F0A0008A086010037B5114B53
:100AE0001A780132D2B20024012A01468DF807405B
:100AF00011D80D4803681D6A4FF47A734B430122E5
:100B00000DF10701A847012805D1084B9DF8070002
:100B10001C7003B030BD4FF4FA7000F01DFF4FF0B1
:100B2000FF30F6E700240020482A00208429002016
:100B300038B50E4B1A780132D2B2012A05460ED8CA
:100B40000B4803681C6A4FF47A734B43042229460E
:100B5000A047042803D1074B0020187038BD4FF47C
:100B6000FA7000F0F9FE4FF0FF3038BD002400208D
:100B7000482A00208429002030B4054C2368DD6910
:100B8000044B0A46AC460146204630BC604700BFD5
:100B9000482A0020A086010070B501F027F9094C11
:100BA000094E2070002530682378834208D901F06F
:100BB00017F9336805440133B5F5803F3360F2D34C
:100BC00070BD00BF852900208029002001F0BCB93C
:100BD00000F1006000F580300068704700F10060AF
:100BE000920000F5803001F047B90000054B1A680B
:100BF000054B1B789B1A834202D9104401F0F0B8D0
:100C000000207047802900208529002038B5074D35
:100C100004462868204401F0EBF828B928682044ED
:100C2000BDE8384001F0FCB838BD00BF8029002085
:100C300010F0030308D1B0F5007F05D800F1005093
:100C4000A0F508400068704700207047014BC0586D
:100C5000704700BF107AFF1F014B1868704700BF34
:100C6000002004E070B52A4B1C68C4F30B03240C6D
:100C700063B140F21342934231D040F219429342A1
:100C80002FD040F2214293422DD10323214A0C253B
:100C900005FB03235D6893F9082042F201039C429F
:100CA00024D0B4F5805F23D041F201039C4221D0CF
:100CB00041F203039C421FD041F207039C4208BF4C
:100CC0003122441E0C44013D0B46A3421ED215F9AD
:100CD000016F581C96B1034600F8016CF5E701233B
:100CE000D4E70223D2E73F220B4DD6E73322E3E7D6
:100CF0004122E1E75A22E4E75922E2E72C25844227
:100D00001D7001D9981C5A70401A70BD1846FBE737
:100D1000002004E008340008FC330008022804D155
:100D2000054B4FF480229A6170470128FCD14FF4A3
:100D30008032024BF7E700BF000C0240000802407F
:100D4000022803D1044B04229A617047012804BF92
:100D5000024B9861704700BF000C0240000802403F
:100D6000022805D1064A536983F004035361704792
:100D70000128FCD1034A536983F00103F6E700BF61
:100D8000000C02400008024010B50023934203D03B
:100D9000CC5CC4540133F9E710BD000030B5441EEB
:100DA00014F9010F0B4660B193F90050854201F12F
:100DB000010106D11AB993F90020801A30BD013A19
:100DC000EEE7002AF7D1104630BD00000246034688
:100DD000981A13F9011B0029FAD1704702440346FF
:100DE000934202D003F8011BFAE77047024B1A78CE
:100DF000024B1A70704700BF842900200024002095
:100E000038B5104D104C284600F0EEF82146284623
:100E100000F016F924680D48626DD2F8043843F0EA
:100E20000203C2F8043800F097FD0949204600F09B
:100E300013FA626DD2F8043823F00203C2F80438C2
:100E400038BD00BF482A0020D434000840420F00BB
:100E5000FC34000870470000FEE7000000B59BB0BE
:100E6000EFF3098168226846FFF78EFFEFF30583F1
:100E7000034B9A6B9A6A9A6A9A6A9A6A9B6AFEE725
:100E800000ED00E000B59BB0EFF3098168226846F1
:100E9000FFF77AFFEFF30583044B9A6B9A6A9A6A1D
:100EA0009A6A9A6A9A6A9B6AFEE700BF00ED00E0C0
:100EB00000B59BB0EFF3098168226846FFF764FF35
:100EC000EFF30583034B5A6B9A6A9A6A9A6A9A6A95
:100ED0009B6AFEE700ED00E0002304491A465A50E1
:100EE000C8180833802B4260F9D170478829002048
:100EF000026843681143016003B11847704700005E
:100F000013B5446BD4F894341A681178042915D1B8
:100F1000217C022912D11979128901238B401342B5
:100F20000CD101A904F14C0001F028FED4F894443E
:100F3000019B21790246206800F0DAF902B010BD69
:100F4000143001F0ABBD00004FF0FF33143001F05E
:100F5000A5BD00004C3001F07DBE00004FF0FF3316
:100F60004C3001F077BE0000143001F079BD000074
:100F70004FF0FF31143001F073BD00004C3001F030
:100F800049BE00004FF0FF324C3001F043BE00007C
:100F9000D0F8942438B5136819780429054601D08F
:100FA000012038BD017C0229FAD112795C89012027
:100FB00090400440F4D105F1140001F00BFD02460D
:100FC0000028EDD0D5F894544FF4807328686979DF
:100FD00000F07CF9204638BD406BFFF7D9BF000018
:100FE00000207047704700007FB5124B036000235C
:100FF00043608360C360012502260F4B05740446DD
:101000000290019300F18402294600964FF4807308
:10101000143001F0BBFC094B0193029400964FF48D
:10102000807304F52372294604F14C0001F082FD1F
:1010300004B070BD58340008D90F0008010F000833
:101040000B68202282F311880A7903EB82029061F7
:101050004A79093243F822008A7912B103EB8203FC
:10106000986102230374C0F89414002383F3118859
:101070007047000038B5037F044613B190F8543030
:10108000ABB9201D01250221FFF732FF04F1140046
:1010900025776FF0010100F087FC84F8545004F1CB
:1010A0004C006FF00101BDE8384000F07DBC38BD58
:1010B00010B5012104460430FFF71AFF00232377FF
:1010C00084F8543010BD000038B5044600251430B3
:1010D00001F074FC04F14C00257701F043FD201D64
:1010E00084F854500121FFF703FF2046BDE8384043
:1010F000FFF74EBF90F8443003F06003202B19D166
:1011000090F84520212A0AD0222A4FF000030ED061
:10111000202A0FD1084A82630722C26304E0064BEB
:1011200083630723C3630023036401207047836341
:10113000C363F9E70020704701240020D0F89434FD
:1011400037B51A681178042904461AD1017C02299E
:1011500017D11979128901238B40134211D100F163
:101160004C05284601F0BEFD58B101A9284601F002
:1011700005FDD4F89444019B21790246206800F0D3
:10118000B7F803B030BD000000EB8103F7B59C69F0
:1011900005460E46F4B1202383F3118805EB86073C
:1011A000201D0821FFF7A4FEFB685B691B684C3417
:1011B00013B1204601F0F0FC01A9204601F0DEFC4D
:1011C000024648B1019B3146284600F091F80023C1
:1011D00083F3118803B0F0BDFB685A691268002AD6
:1011E000F5D01B8A013B1340F1D105F14402EAE737
:1011F000093138B550F82140DCB1202383F3118840
:10120000D4F894241368527903EB8203DB689B695A
:101210005D6845B104216018FFF76AFE294604F1B4
:10122000140001F0E1FB2046FFF7B2FE002383F338
:10123000118838BD7047000000F08CBF0123037097
:1012400000234360C36183620362C362436203633A
:10125000038143817047000038B50446202383F39F
:10126000118800254160C56005614561856100F018
:1012700081FF0223237085F3118838BD70B500EB20
:10128000810305465069DA600E46144618B11022F3
:101290000021FFF7A3FDA06918B110220021FFF77C
:1012A0009DFD31462846BDE8704001F02DB8000094
:1012B000028902F001020281428902F001024281A8
:1012C000002202614261826101F0B2B8F0B400EB29
:1012D00081044789E4680125A4698D403D43458127
:1012E00023600023A2606360F0BC01F0CDB8000071
:1012F000F0B400EB81040789E468012564698D403E
:101300003D43058123600023A2606360F0BC01F0CF
:1013100047B9000070B50223002504460370A0F809
:101320004C5080F84E5080F84F5005814581C56083
:1013300005614561856180F8345000F081FF636884
:101340001B6823B129462046BDE87040184770BD90
:10135000436802781B6880F85020052202700BB1A8
:101360000421184770470000436890F850201B681C
:1013700002700BB1052118477047000090F8343017
:1013800070B5044613B1002380F8343004F14402F0
:10139000204601F06FF863689B6863BB94F8445083
:1013A00015F0600615D194F8453005F07F0545EA43
:1013B000032540F202339D4200F00E815BD8022DDE
:1013C00000F0DC803FD8002D00F08780012D00F078
:1013D000CF800021204601F0A5FA0021204601F02F
:1013E00097FA63681B6813B10621204698470623C5
:1013F00084F8343070BD204698470028CED094F849
:101400004B2094F84A3043EA0223E26B934238BF00
:10141000E36394F94430E56B002B4FF0200380F236
:10142000FD80002D00F0EC80092284F8342083F345
:1014300011880021E36BA26B2046FFF759FF0023C0
:1014400083F3118870BDB5F5817F00F0B180B5F5EB
:10145000407F49D0B5F5807FBBD194F84630012B51
:10146000B7D1B4F84C3023F00203A4F84C30A66393
:10147000E6632664C3E740F201639D421ED8B5F5DA
:10148000C06F3BD2B5F5A06FA3D1B4F84430B3F52B
:10149000A06F0ED194F8463084F84E30204600F00C
:1014A00027FF63681B6813B1012120469847032377
:1014B00023700023A363E3632364A0E7B5F5106FF3
:1014C00032D040F602439D4252D0B5F5006F80D134
:1014D00004F14F03A363012324E004F14C03A3634D
:1014E0000223E36325648AE794F84630012B7FF4F6
:1014F00070AFB4F84C3043F00203B6E794F84920DB
:10150000616894F848304D6894F8471043EA022324
:10151000204694F84620A84700283FF45AAF436875
:10152000A3630368E363A4E72378042B10D120238B
:1015300083F311882046FFF7BBFE86F311886368AA
:1015400084F84F601B68032121700BB12046984737
:1015500094F84630002BACD084F84F30042323702D
:1015600063681B68002BA4D0022120469847A0E79F
:10157000374BA3630223E36300239DE794F84810ED
:1015800011F0800F204601F00F010ED000F064FF33
:10159000012806D002287FF41CAF2E4BA363E06322
:1015A00067E72D4BA363E56363E700F047FFEFE7D1
:1015B00094F84630002B7FF40CAF94F8483013F0C9
:1015C0000F013FF476AF1A06204602D501F0BEF9AE
:1015D0006FE701F0B1F96CE794F84630002B7FF427
:1015E000F8AE94F8483013F00F013FF462AF1B06D9
:1015F000204602D501F096F95BE701F089F958E73A
:10160000142284F8342083F311882B462A46294675
:101610002046FFF75BFE85F3118870BD5DB1152292
:1016200084F8342083F311880021E36BA26B2046F9
:10163000FFF74CFE03E70B2284F8342083F3118874
:101640002B462A4629462046FFF752FEE3E700BF15
:1016500088340008803400088434000838B590F8D5
:1016600034300446152B29D8DFE803F03E2828281B
:1016700028283E28280B29392828282828282828DF
:101680003E3E90F84B1090F84A20C36B42EA01228C
:101690009A4214D9C268128AB3FBF2F502FB1535DF
:1016A0006DB9202383F311882B462A462946FFF77C
:1016B0001FFE85F311880A2384F8343038BD1423C3
:1016C00084F83430202383F3118800231A46194606
:1016D0002046FFF7FBFD002383F3118838BD036C20
:1016E00003B198470023E7E7002101F01BF900212F
:1016F000204601F00DF963681B6813B106212046EE
:1017000098470623D8E7000090F83420152A38B50A
:10171000044622D80123934040F6416213421DD172
:1017200013F480150FD19B0217D50B2380F83430AA
:10173000202383F311882B462A462946FFF7D8FD3C
:1017400085F3118838BDC3689B695B682BB9036C4E
:1017500003B19847002384F8343038BD002101F0EC
:10176000E1F80021204601F0D3F863681B6813B14B
:101770000621204698470623EDE70000024B002291
:101780001B605B609A607047082A00200023037486
:101790008268054B1B6899689142FBD25A680360C6
:1017A0004260106058607047082A002008B5202366
:1017B00083F31188037C032B05D0042B0DD02BB9A8
:1017C00083F3118808BD436900221A604FF0FF338C
:1017D0004361FFF7DBFF0023F2E790E80C001A609B
:1017E00002685360F2E70000002303748268054B2F
:1017F0001B6899689142FBD85A6803604260106088
:1018000058607047082A0020054B19690874186849
:1018100002681A605360186101230374FEF774BDF7
:10182000082A002030B54B1C87B005460A4C10D062
:1018300023690A4A01A800F0D3F82846FFF7E4FF1D
:10184000049B13B101A800F007F92369586907B098
:1018500030BDFFF7D9FFF8E7082A0020AD170008D0
:1018600038B50C4D41612B6981689A6891420446F4
:1018700003D8BDE83840FFF789BF1846FFF786FF59
:1018800001232C61014623742046BDE83840FEF751
:101890003BBD00BF082A0020044B1A681B699068F2
:1018A0009B68984294BF002001207047082A0020BE
:1018B00010B5084C236820691A6822605460012220
:1018C00023611A74FFF790FF01462069BDE81040BC
:1018D000FEF71ABD082A002082600222027400224C
:1018E000427470478368A3F17C0243F80C2C0269B0
:1018F00043F83C2C426943F8382C074A43F81C2C27
:10190000C26843F8102C022203F8082C002203F8C6
:10191000072CA3F1180070472103000810B52023FD
:1019200083F31188FFF7DEFF00210446FFF798FFDD
:10193000002383F31188204610BD0000024B1B6971
:1019400058610F20FFF760BF082A0020202383F38F
:101950001188FFF7F3BF000008B50146202383F389
:1019600011880820FFF75EFF002383F3118808BD6C
:1019700049B1064B42681B6918605A6013604360A6
:101980000420FFF74FBF4FF0FF307047082A0020B8
:101990000368984206D01A68026050605961184680
:1019A000FFF7F4BE7047000038B504460D462068C6
:1019B000844200D138BD036823605C604561FFF755
:1019C000E5FEF4E7054B03F114025A619A614FF00A
:1019D000FF32DA6100221A62704700BF082A002035
:1019E000F8B503611A4BC2605C6A1A4B1A460229A9
:1019F00052F8145F38BF0221954206461F460AD1AD
:101A0000586198611C620560456081600819BDE8F5
:101A1000F84001F089B9186AAB68241A0C1902D38E
:101A2000E41A2D6804E09C4202D2204401F08CF9B3
:101A3000AB689C42F4D86B68736035601E606E6062
:101A4000B460A9684FF0FF33091BA960FB61F8BDC2
:101A5000000C0040082A002010B41A4C234653F80A
:101A6000141F814210D0416802680A600268516008
:101A70009A424FF00001C16003D0936881680B4423
:101A800093605DF8044B70470A68626100209A42D7
:101A90005360C86003D15DF8044B01F04FB99368FF
:101AA000886803449360084A206A526A121A934273
:101AB000E7D9991A012998BF931C18445DF8044B83
:101AC00001F042B9082A0020000C004000207047B5
:101AD000FEE70000704700004FF0FF307047000045
:101AE000022906D0032906D00129064818BF002084
:101AF000704705487047032A9ABF044800EBC200AC
:101B000000207047583500080C35000808240020D4
:101B100070B59AB001AD064608462946144600F055
:101B200095F82846FFF752F9C0B2431C5B0086E8DF
:101B30001800237003236370002302341946DAB2BD
:101B4000904204F1020401D81AB070BDEA5C04F8B6
:101B5000022C04F8011C0133F1E7000008B5202332
:101B600083F311880348FFF7E9FA002383F3118810
:101B700008BD00BF482A002010B50446052916D824
:101B8000DFE801F016150316161D202383F31188D4
:101B90000E4A0121FFF772FB20460D4A0221FFF792
:101BA0006DFB0C48FFF790FA002383F3118810BDFA
:101BB000202383F311880748FFF75CFAF4E720231A
:101BC00083F311880348FFF773FAEDE78C340008BC
:101BD000B0340008482A002038B50C4D0C4C0D4993
:101BE0002A4604F10800FFF793FF05F1CA0204F149
:101BF00010000949FFF78CFF05F5CA7204F11800BF
:101C00000649BDE83840FFF783BF00BF102F002012
:101C100008240020DC340008E6340008F134000811
:101C200070B5044608460D46FFF7D0F8C6B2204608
:101C3000013403780BB9184670BD32462946FFF7C8
:101C4000ADF80028F3D1012070BD00002DE9F84F58
:101C500005460C46FFF7BAF82B49C6B22846FFF7EF
:101C6000DFFF08B10336F6B228492846FFF7D8FF50
:101C700008B11036F6B2632E0DD8DFF88C80DFF88D
:101C80008C90234FDFF890A0DFF890B02E7846B903
:101C90002670BDE8F88F29462046BDE8F84F01F0D0
:101CA000A1BB252E2CD1072241462846FFF776F806
:101CB00058B9DBF800302360DBF804306360BBF810
:101CC0000830238107350A34E0E7082249462846D0
:101CD000FFF764F8A0B90F4BA21C13F8011F090904
:101CE0005345C95D02F8021C197801F00F0102F199
:101CF0000202C95D02F8031CEFD118340835C5E7AC
:101D0000267001350134C1E778350008F134000848
:101D10008B3500080F7AFF1F1B7AFF1F80350008E4
:101D2000BFF34F8F024AD368DB03FCD4704700BF78
:101D3000003C024008B5094B1B7873B9FFF7F0FF70
:101D4000074B1A69002ABFBF064A5A6002F188325F
:101D50005A601A6822F480621A6008BD6E31002051
:101D6000003C02402301674508B50B4B1B7893B933
:101D7000FFF7D6FF094B1A6942F000421A611A6850
:101D800042F480521A601A6822F480521A601A686B
:101D900042F480621A6008BD6E310020003C0240AF
:101DA0000B2870B513D80B4A0B4C137863B90B4E44
:101DB0004FF0006144F8231056F8235001330C2BE8
:101DC0002944F7D10123137054F8200070BD00207E
:101DD00070BD00BFA0310020703100209C3500088C
:101DE000014B53F8200070479C3500080C207047C9
:101DF0000B2810B5044601D9002010BDFFF7D0FF15
:101E0000064B53F824301844C21A0BB9012010BDF8
:101E100012680132F0D1043BF6E700BF9C350008A0
:101E20000B2810B5044621D8FFF77AFFFFF782FF91
:101E30000F4AF323D360C300DBB243F4007343F0D3
:101E400002031361136943F480331361FFF768FFE2
:101E5000FFF7A6FF074B53F8241000F0DDF8FFF75B
:101E600083FF2046BDE81040FFF7C2BF002010BD31
:101E7000003C02409C3500082DE9F84312F00103B4
:101E8000154640D18218B2F1016F3CD22C4B1B6831
:101E900013F0010337D02B4CFFF74CFFF323E36023
:101EA000FFF73EFF40F20127032D01D9830713D02E
:101EB000244C0F46401A40F20118EB1B0B44012B37
:101EC00000EB0706236924D823F001032361FFF701
:101ED0004BFF0120BDE8F883236923F4407323619D
:101EE00023693B43236151F8046B0660BFF34F8FB6
:101EF000FFF716FF03689E4208D0236923F0010311
:101F00002361FFF731FF0020BDE8F883043D043072
:101F1000CAE723F440732361236943EA080323617A
:101F2000B94637F8023B3380BFF34F8FFFF7F8FE17
:101F30003688B9F80030B6B2B342BED0DDE700BF94
:101F400000380240003C0240084908B50B7828B12F
:101F500053B9FFF7EFFE01230B7008BD23B1BDE8B5
:101F600008400870FFF700BF08BD00BF6E310020B9
:101F700010B50244064B0439D2B2904200D110BDD4
:101F8000441C00B253F8200041F8040FE0B2F4E71B
:101F900050280040104B30B51C6F240407D41C6F30
:101FA00044F400741C671C6F44F400441C670B4C21
:101FB000236843F4807323600244094B0439D2B28E
:101FC000904200D130BD441C00B251F8045F43F888
:101FD0002050E0B2F4E700BF00380240007000403B
:101FE0005028004007B5012201A90020FFF7C0FFDB
:101FF000019803B05DF804FB13B50446FFF7F2FF48
:10200000A04206D002A9012241F8044D0020FFF7AA
:10201000C1FF02B010BD000070470000034B1B68F9
:102020009B0042BF024B01221A7070477438024075
:10203000A1310020014B1878704700BFA13100206A
:1020400070470000FEE70000084A094B09498B422F
:1020500004D3094A0021934205D3704752F8040F74
:1020600043F8040BF3E743F8041BF4E74437000894
:10207000183400201834002018340020836D30B547
:1020800000229D68446D11464FF0FF3004EB42136F
:1020900001329542C3F80019C3F81019C3F80809B2
:1020A000C3F8001BC3F8101BC3F8080BEED24FF0A7
:1020B0000113C4F81C3830BD890141F020010161D1
:1020C00003699B06FCD4122000F0CABE204B03EB30
:1020D00080022DE9F047D2F80CE05D6DDEF81420A7
:1020E000461CD2F800C005EB063605EB40185168D7
:1020F00061450BD3D5F83428012303FA00F022EA16
:102100000000C5F834081846BDE8F087BEF8104056
:10211000ACEB0103A34228BF2346D8F81849A4B268
:10212000B3EB840F10D894681F46A4F1040959F842
:1021300004AFC6F800A0042F01D9043FF7E71C4400
:102140000B4494605360D2E70020BDE8F08700BFE5
:10215000A431002010B5054C2046FFF76FF84FF072
:10216000A0436365024BA36510BD00BFA4310020EE
:10217000F03500080378012B70B5054650D12A4B85
:10218000446D98421BD1294B5A6B42F080025A632E
:102190005A6D42F080025A655A6D5A6942F08002C7
:1021A0005A615A6922F080025A610E2143205B690C
:1021B00000F0D6FB1E4BE3601E4BC4F80038002332
:1021C000C4F8003EC02323606E6D4FF40413A36374
:1021D0003369002BFCDA012333610C2000F040FE50
:1021E0003369DB07FCD4122000F03AFE3369002B80
:1021F000FCDA0026A6602846FFF740FF6B68C4F8AB
:102200001068DB68C4F81468C4F81C684BB90A4B42
:10221000A3614FF0FF336361A36843F00103A36040
:1022200070BD064BF4E700BFA43100200038024027
:102230004014004003002002003C30C0083C30C085
:10224000F8B5446D054600212046FFF735FFA96D1E
:1022500000234FF001128F68C4F834384FF0006645
:10226000C4F81C284FF0FF3004EB431201339F42A7
:10227000C2F80069C2F8006BC2F80809C2F8080B7E
:10228000F2D20B686A6DEB65636210231361166905
:1022900016F01006FBD1122000F0E2FDD4F8003851
:1022A00023F4FE63C4F80038A36943F4402343F0E9
:1022B0001003A3610923C4F81038C4F814380A4B7A
:1022C000EB604FF0C043C4F8103B084BC4F8003B30
:1022D000C4F81069C4F80039EB6D03F1100243F43F
:1022E0008013EA65A362F8BDCC3500084080001079
:1022F000426D90F84E10D2F8003823F4FE6343EAA2
:102300000113C2F8003870472DE9F0410EB200EB1E
:1023100086080D46D8F80C100F6807F00303022B4F
:1023200050D0032B50D03D4A3D4F012B18BF1746CC
:10233000446D4FEA451E04EB0E030022C3F8102B38
:102340008A6905F1100C002A40D04A8A05F1580329
:102350005B013A43E2500123D4F81C2803FA0CF342
:102360001343A6444A69C4F81C380023CEF8103938
:1023700005F13F03002A39D00A8A898B9208012986
:1023800088BF4A43C16D04EB8303561841EA0242F9
:10239000C66529465A602046FFF78EFED8F80C30F5
:1023A0001B8A43EA85531F4305F148035B01E7504D
:1023B0000123D4F81C2803FA05F51543C4F81C586A
:1023C000BDE8F081174FB3E7174FB1E704EB4613B1
:1023D000D3F8002B22F40042C3F8002BD4F81C28B9
:1023E000012303FA0CF322EA0303BAE704EB8303A5
:1023F0000E4A5A6004EB461629462046FFF75CFE5B
:10240000D6F8003923F40043C6F80039D4F81C3854
:10241000012202FA05F523EA0505CFE70080001046
:10242000008004100080081000800C1000040002DE
:10243000826D1268C265FFF721BE00005831436DFE
:1024400049015B5813F4004004D013F4001F14BF7B
:1024500001200220704700004831436D49015B585C
:1024600013F4004004D013F4001F14BF0120022015
:102470007047000000EB8101CB68196A0B6813609C
:102480004B6853607047000000EB810330B5DD6896
:10249000AA691368D36019B9402B84BF4023136025
:1024A0006B8A1468426D1C44013CB4FBF3F4634333
:1024B000033323F0030302EB411043EAC44343F028
:1024C000C043C0F8103B2B6803F00303012B09B293
:1024D0000ED1D2F8083802EB411013F4807FD0F807
:1024E000003B14BF43F0805343F00053C0F8003B5F
:1024F00002EB4112D2F8003B43F00443C2F8003B28
:1025000030BD00002DE9F041244D6E6D06EB401307
:102510000446D3F8087BC3F8087B38070AD5D6F8F9
:102520001438190706D505EB84032146DB682846D5
:102530005B689847FA072FD5D6F81438DB072BD5F8
:1025400005EB8403D968CCB98B69488A5E68B6FB11
:10255000F0F200FB12628AB91868DA6890420DD274
:10256000121A83E81400202383F311880B482146B4
:10257000FFF78AFF84F31188BDE8F081012303FA95
:1025800004F26B8923EA02036B81CB6823B12146F5
:102590000248BDE8F0411847BDE8F081A4310020B1
:1025A00000EB810370B5DD68436D6C692668E660F9
:1025B0004A0156BB1A444FF40020C2F810092A6899
:1025C00002F00302012A0AB20ED1D3F8080803EB85
:1025D000421410F4807FD4F8000914BF40F08050FA
:1025E00040F00050C4F8000903EB4212D2F8000991
:1025F00040F00440C2F80009D3F83408012202FA7E
:1026000001F10143C3F8341870BD19B9402E84BFDD
:102610004020206020682E8A841940F00050013C40
:102620001A44B4FBF6F440EAC440C6E7F8B50446E1
:102630001E48456D05EB4413D3F80869C3F80869D3
:10264000F10717D5D5F81038DA0713D500EB840356
:10265000D9684B691F68DA68974218D2D21B0027E5
:102660001A605F60202383F311882146FFF798FFEB
:1026700087F31188330617D5D5F834280123A340F2
:10268000134211D02046BDE8F840FFF71FBD0123DB
:1026900003FA04F2038923EA020303818B68002B07
:1026A000E8D021469847E5E7F8BD00BFA4310020F7
:1026B00096482DE9F84F456D6E69AB691E4016F4DA
:1026C000805F6E61044605D0FEF724FEBDE8F84F3A
:1026D00000F05ABC002E12DAD5F8003E8B489B075A
:1026E0001EBFD5F8003E23F00303C5F8003ED5F821
:1026F000043823F00103C5F80438FEF735FE37052A
:1027000002D58248FEF724FEB0040CD5D5F808386F
:1027100013F0060FEB6823F470530CBF43F410530F
:1027200043F4A053EB60310704D56368DB680BB159
:1027300076489847F2025AD4B3020CD5D4F85480A4
:10274000DFF8C8A100274FF00109A36D9B68F9B21B
:102750008B4280F08780F70619D5616D0A6AC2F353
:102760000A1702F00F0302F4F012B2F5802F00F006
:10277000A180B2F5402F0AD104EB830301F580510B
:10278000DB68186A00231A469F4240F087803003B6
:10279000D5F8184813D5E10302D50020FFF7B2FEA3
:1027A000A20302D50120FFF7ADFE630302D502208C
:1027B000FFF7A8FE270302D50320FFF7A3FE75034A
:1027C00084D5E00702D50020FFF730FFA10702D52E
:1027D0000120FFF72BFF620702D50220FFF726FF3B
:1027E00023077FF573AF0320FFF720FF6EE7D4F8D0
:1027F0005480DFF818A100274FF00109A36D9B68F2
:102800005FFA87FB5B4597D308EB4B13D3F800299E
:1028100002F44022B2F5802F22D1D3F80029002AF9
:102820001EDAD3F8002942F09042C3F80029D3F809
:102830000029002AFBDB5946606DFFF73DFC228929
:1028400009FA0BF322EA0303238104EB8B03DB6811
:102850009B6813B15946504698475846FFF736FCD7
:102860000137CBE708EB4112D2F8003B03F44023D9
:10287000B3F5802F10D1D2F8003B002B0CDA62891F
:1028800009FA01F322EA0303638104EB8103DB68A5
:10289000DB680BB150469847013756E79C0708BFE5
:1028A0000A68072B98BF027003F101039CBF120A4C
:1028B000013069E7023304EB830201F5805152686D
:1028C00090690268D0F808C04068A2EB000E0022B0
:1028D000104697420AD104EB830463689B699A68A7
:1028E0003A449A605A6817445F6050E712F0030F49
:1028F00008BF0868964588BF8CF8000002F1010205
:1029000084BF000A0CF1010CE3E700BFA4310020F2
:10291000436D03EB4111D1F8003B43F40013C1F8C0
:10292000003B7047436D03EB4111D1F8003943F48C
:102930000013C1F800397047436D03EB4111D1F822
:10294000003B23F40013C1F8003B7047436D03EBD9
:102950004111D1F8003923F40013C1F80039704750
:1029600000F1604300F01F02400903F561430901D3
:102970008000C9B200F1604083F8001300F56140A7
:1029800001239340C0F880310360704730B5039C49
:102990000172043304FB0325C361049B036300211C
:1029A000059B00604060C160426102618561046214
:1029B00042628162C162436330BD00000022416A0D
:1029C00041610161C2608262C2626FF00101FEF783
:1029D000EBBF000003694269934203D1C2680AB1A8
:1029E00000207047181D704703691960C2680132E2
:1029F000C260C269134482690361934224BF436A7F
:102A000003610021FEF7C4BF38B504460D46E368F4
:102A10003BB16269131D1268A3621344E362002094
:102A200038BD237A33B929462046FEF7A1FF002896
:102A3000EDDA38BD6FF00100FBE70000C368C26942
:102A4000013BC3604369134482694361934224BFDD
:102A5000436A436100238362036B03B118477047E5
:102A600070B52023044683F31188866A3EB9FFF7C8
:102A7000CBFF054618B186F31188284670BDA36ABE
:102A8000E26A13F8015BA362934202D32046FFF788
:102A9000D5FF002383F31188EFE700002DE9F84FFD
:102AA00004460E4690469946202787F31188002554
:102AB000AA46D4F828B0BBF1000F09D149462046F8
:102AC000FFF7A2FF20B18BF311882846BDE8F88FED
:102AD000A16AE36AA8EB050B5B1A9B4528BF9B46DE
:102AE000BBF1400F1BD9334601F1400251F8040BF2
:102AF00043F8040B9142F9D1A36A40334036A362F4
:102B00004035A26AE36A9A4202D32046FFF796FF55
:102B10008AF311884545D8D287F31188C9E7304632
:102B20005A46FEF731F9A36A5B445E44A3625D44F2
:102B3000E7E7000010B5029C0172043303FB042197
:102B4000C36100238362C362039B0363049B006031
:102B50004060C46042610261816104624262436319
:102B600010BD0000026AC260426A42610261002236
:102B70008262C2626FF00101FEF716BF436902690B
:102B80009A4203D1C2680AB100207047184650F833
:102B9000043B0B6070470000C368C2690133C36027
:102BA0004369134482694361934224BF436A43618A
:102BB0000021FEF7EDBE000038B504460D46E3687F
:102BC0003BB123691A1DA262E2691344E36200204B
:102BD00038BD237A33B929462046FEF7C9FE0028BE
:102BE000EDDA38BD6FF00100FBE700000369196002
:102BF000C268013AC260C2691344826903619342A8
:102C000024BF436A036100238362036B03B1184747
:102C10007047000070B5202304460E4683F31188E8
:102C2000856A35B91146FFF7C7FF10B185F31188E2
:102C300070BDA36A1E70A36AE26A01339342A36265
:102C400004D3E16920460439FFF7D0FF002080F368
:102C5000118870BD2DE9F84F04460D4691469A46FD
:102C60004FF0200888F311880026B346A76A4FB9B1
:102C700051462046FFF7A0FF20B187F31188304668
:102C8000BDE8F88FA06AE76AA9EB06033F1A9F42E6
:102C900028BF1F46402F1BD905F1400355F8042BD0
:102CA00040F8042B9D42F9D1A36A4033A362403619
:102CB000A26AE36A9A4204D3E16920460439FFF725
:102CC00095FF8BF311884E45D9D288F31188CDE753
:102CD00029463A46FEF758F8A36A3B443D44A362AE
:102CE0003E44E5E7026943699A4203D1C3681BB9D0
:102CF000184670470023FBE7836A002BF8D0043B9B
:102D00009B1AF5D01360C368013BC360C3691A44C2
:102D1000836902619A4224BF436A0361002383628C
:102D20000123E5E700F072B9034B002258631A61F2
:102D30000222DA60704700BF000C0040014B002205
:102D4000DA607047000C0040014B5863704700BFC9
:102D5000000C0040FEE7000010B5174CFEF70EFD1A
:102D6000FEF730FE802215492046FEF7B5FD01230F
:102D700044F8180C0374124B124AD96821F4E0612C
:102D80000904090C0A431049DA60CA6842F08072EB
:102D9000CA600E490A6842F001020A601022DA771E
:102DA000202283F82220002383F3118862B608488A
:102DB000BDE81040FEF7B2BD302A0020FC35000807
:102DC00000ED00E00003FA05F0ED00E0001000E087
:102DD000043600082DE9F84F1F4CDFF88090656934
:102DE00004F114074FF00008D9F82430266AAA68C5
:102DF0009E1B96421DD34FF0200AAA68236AD5F87D
:102E00000CB0134423622B68BB425F60A6EB020642
:102E10006361C5F80C8001D1FFF790FF88F311883A
:102E20002869D8478AF311886569AB689E42E4D265
:102E3000DAE76269BA420CD0916823628E1B966011
:102E4000A86802282CBF1818981CBDE8F84FFFF797
:102E50007BBFBDE8F88F00BF082A0020000C0040AF
:102E6000034B59685A68521A9042FBD8704700BF0A
:102E7000001000E04B6843608B688360CB68C360E0
:102E80000B6943614B6903628B6943620B680360A2
:102E90007047000008B5224B22481A6940F2FF1122
:102EA0000A431A611A6922F4FF7222F001021A61C0
:102EB0001A691A6B0A431A631A6D0A431A651A4A89
:102EC0001B6D1146FFF7D6FF184802F11C01FFF7F2
:102ED000D1FF174802F13801FFF7CCFF154802F186
:102EE0005401FFF7C7FF144802F17001FFF7C2FF5A
:102EF000124802F18C01FFF7BDFF114802F1A80151
:102F0000FFF7B8FF0F4802F1C401FFF7B3FF0E4807
:102F100002F1E001FFF7AEFFBDE8084000F0E2B8C3
:102F2000003802400000024024360008000402403D
:102F300000080240000C0240001002400014024051
:102F400000180240001C02400020024008B500F0BA
:102F500039FAFFF701FFFFF761F8BDE80840FEF717
:102F60003BBE000070470000064A536823F001038F
:102F70005360EFF30983683383F30988002383F3F5
:102F80001188704730EF00E010B5202383F31188DB
:102F9000104B5B6813F4006318D0F1EE103AEFF3B6
:102FA00009844FF0807344F84C3C0B4BDB6844F8C9
:102FB000083CA4F1680383F30988FEF76DFC18B19F
:102FC000064B44F8503C10BD054BFAE783F31188DB
:102FD00010BD00BF00ED00E030EF00E0310300085D
:102FE00034030008084B1A69920710B508D500246D
:102FF0001C61202383F31188FFF7ECFE84F3118812
:10300000BDE81040FFF7C0BF000C0040104B1A6C29
:1030100042F008021A641A6E42F008021A660D4A5B
:103020001B6E936843F0080393600B4B53229A6224
:103030004FF0FF32DA6200229A615A63DA605A6016
:1030400001225A6108211A603220FFF789BC00BFB3
:1030500000380240002004E0000C00401F4B1A69B9
:103060006FEAC2526FEAD2521A611A69C2F30802B9
:103070001A614FF0FF301A695A69586100215A6984
:1030800059615A691A6A62F080521A621A6A02F029
:1030900080521A621A6A5A6A58625A6A59625A6A9D
:1030A0001A6C42F080521A641A6E42F080521A660C
:1030B0001A6E0B4A106840F480701060186F00F4AC
:1030C0004070B0F5007F1EBF4FF48030186719675D
:1030D000536823F40073536000F054B90038024081
:1030E00000700040304B4FF080521A642F4A4FF46A
:1030F000404111601A6842F001021A601A68920792
:10310000FCD59A6822F003029A60274B19469A6808
:1031100012F00C02FBD1186800F0F90018609A60F8
:103120001A6842F480321A600B689B03FCD54B6F1F
:1031300043F001034B671C4B5A6F9007FCD51C4AA8
:103140005A601A6842F080721A60184A536859042B
:10315000FCD5154B1A689201FCD5164A9A60164B9D
:103160001A68164B9A42164B1BD1164A1168164A1A
:10317000914216D140F205121A600B4B9A6842F048
:1031800002029A609A6802F00C02082AFAD15A6C7C
:1031900042F480425A645A6E42F480425A665B6E30
:1031A000704740F20572E7E70038024000700040C7
:1031B0000854400700948838002004E0116400207F
:1031C000003C024000ED00E041C20F41084A08B552
:1031D000536911680B4003F00103536123B1054AA1
:1031E00013680BB150689847BDE80840FFF7CCBEA4
:1031F000003C014088290020084A08B5536911683D
:103200000B4003F00203536123B1054A93680BB1ED
:10321000D0689847BDE80840FFF7B6BE003C0140C3
:1032200088290020084A08B5536911680B4003F04B
:103230000403536123B1054A13690BB150699847E0
:10324000BDE80840FFF7A0BE003C014088290020EF
:10325000084A08B5536911680B4003F0080353612D
:1032600023B1054A93690BB1D0699847BDE808407E
:10327000FFF78ABE003C014088290020084A08B5B3
:10328000536911680B4003F01003536123B1054AE1
:10329000136A0BB1506A9847BDE80840FFF774BE47
:1032A000003C014088290020174B10B55C691A6862
:1032B000144004F478725A61A30604D5134A936A41
:1032C0000BB1D06A9847600604D5104A136B0BB156
:1032D000506B9847210604D50C4A936B0BB1D06B09
:1032E0009847E20504D5094A136C0BB1506C984716
:1032F000A30504D5054A936C0BB1D06C9847BDE883
:103300001040FFF741BE00BF003C0140882900206B
:103310001A4B10B55C691A68144004F47C425A6177
:10332000620504D5164A136D0BB1506D98472305FD
:1033300004D5134A936D0BB1D06D9847E00404D5C2
:103340000F4A136E0BB1506E9847A10404D50C4A76
:10335000936E0BB1D06E9847620404D5084A136F80
:103360000BB1506F9847230404D5054A936F0BB1F6
:10337000D06F9847BDE81040FFF706BE003C014003
:1033800088290020062108B50846FFF7E9FA06213A
:103390000720FFF7E5FA06210820FFF7E1FA0621EA
:1033A0000920FFF7DDFA06210A20FFF7D9FA0621E6
:1033B0001720FFF7D5FA06212820BDE80840FFF7BF
:1033C000CFBA000008B5FFF749FEFDF785FDFDF710
:1033D00033FFFDF707FEFFF7C5FDBDE80840FFF727
:1033E000A1BC0000034611F8012B03F8012B002AB1
:1033F000F9D17047121012131211000053544D33BB
:1034000032463F3F3F00000000000000FC33000850
:103410003F00000013040000383400083F000000A3
:1034200019040000423400083F000000210400009D
:103430004C3400083F00000053544D3332463430C2
:10344000780053544D3332463432780053544D3360
:103450003246343436585800000000005D0F000832
:10346000490F0008850F0008710F00087D0F000844
:10347000690F0008550F0008410F0008E10F000810
:103480000000000001000000000000000200000039
:103490000000000089110008F11100084000400000
:1034A000E02E0020F02E00200200000000000000AE
:1034B00003000000000000003512000800000000BA
:1034C00010000000002F002000000000010000009C
:1034D00000000000A4310020010102004172647567
:1034E00050696C6F740025424F415244252D424C67
:1034F000002553455249414C25000000791B000826
:10350000E11A0008F51000085D1B000843000000E8
:103510001435000809024300020100C0320904000A
:103520000001020201000524001001052401000130
:10353000042402020524060001070582030800FF97
:1035400009040100020A0000000705010240000012
:1035500007058102400000001200000060350008ED
:1035600012011001020000408304405700020102D2
:10357000030100000403090425424F415244250081
:103580006372617A79666C69653200303132333446
:103590003536373839414243444546000040000043
:1035A000004000000040000000400000000001005A
:1035B0000000020000000200000002000000020003
:1035C00000000200000002000000020000000000F5
:1035D0007D1300085D160008091700084000400030
:1035E00004320020043200200100000014320020C8
:1035F0008000000040010000030000006D61696E62
:10360000000000001C360008203200201834002082
:1036100001000000552D00080000000069646C6581
:10362000000000000000800200000000AAAAAAAA70
:1036300000000000FFFF00000000000000A00A00E2
:103640000000000000000000AAAAAAAA00000000D2
:10365000FFFF00000000000000000000010000006B
:1036600000000000AAAAAAAA00000000FFFF0000B4
:10367000000000000000000010000000000000003A
:10368000AAAAAAAA00000000FFFF00000000000094
:10369000000000000000000000000000AAAAAAAA82
:1036A00000000000FFFF000000000000000000001C
:1036B0000000000000000000AAAAAAAA0000000062
:1036C000FFFF0000000000000000000000000000FC
:1036D00000000000AAAAAAAA00000000FFFF000044
:1036E00000000000000000000000000000000000DA
:1036F0000A000000000000000300000000000000BD
:1037000000000000000000000000000000000000B9
:1037100000000000000000000000000000000000A9
:10372000FF00960000000008040000007435000847
:103730000000000000000000000000000000000089
:08374000000000000000000081
:00000001FF
